S0120000455642555F5465737465722E733139DA
S11310408E7FFFBD16CFCE210D18CE40012008A6FD
S11310500018A7000818088C210E25F3CC000027DF
S11310600BCE40026F000883000126F88D09BD16DF
S1131070D020FB1046105C34CE10391C0080CC16F6
S1131080D1BD15B9CC16FABD15B9CC1720BD15B90B
S1131090CC1722BD15B9CC174BBD15B9CC1720BD43
S11310A015B9CC177DBD15B9CC17AFBD15B9CC1783
S11310B020BD15B9CC17EABD15B9CC182FBD15B98B
S11310C0CC185FBD15B9CC189CBD15B9CC1720BD83
S11310D015B9CC18E0BD15B9CC192BBD15B9CC196F
S11310E02EBD15B9CC1937BD15B9CC1942BD15B9EA
S11310F0CC1950BD15B9CC1967BD15B9CC198BBD28
S113110015B9CC1720BD15B9BD159DBD163B30E7EB
S1131110004F1A83006527342E281A830061271D87
S1131120CC192BBD15B930E600C17126B1CC199587
S1131130BD15B9CE10391D00804F5F3139BD150C76
S113114020DE1A83007026D88D0920D48D05BD15A4
S11311500C20CDCC19C6BD15B9CC1A01BD15B9CC1E
S113116007D0BD14E4CC1A3ABD15B9C6013734CE44
S113117010003CC6103734CC1000BD138BCC1A7948
S1131180BD15B9C6023734CE10003CC6103734CC76
S11311901000BD138BCC1AB8BD15B9C6043734CEB4
S11311A010003CC6103734CC1000BD138BCC1AF79A
S11311B0BD15B9C6013734CE100A3CC6203734CC2D
S11311C01000BD138BCC1B36BD15B9C6023734CE07
S11311D0100A3CC6203734CC1000BD138BCC1B75D1
S11311E0BD15B9C6043734CE100A3CC6203734CCFA
S11311F01000BD138B30C6243A35CC1BB4BD15B9D1
S1131200C6083734CE100A3CC6203734CC1000BD93
S1131210138BCC1BF3BD15B9C6103734CE100A3C62
S1131220C6403734CC1000BD138BCC1C32BD15B96D
S1131230C6203734CE100A3CC6403734CC1000BD2B
S1131240138BCC1C71BD15B9C6403734CE100A3C83
S11312503734CC1000BD138BCC1CB0BD15B9C6807F
S11312603734CE100A3CC6403734CC1000BD138B43
S1131270CC192BBD15B9CC1CEFBD15B9CC1D26BDA1
S113128015B9CC07D0BD14E4CC1D5DBD15B9CE1085
S1131290091D00041C0008C6043734CE10083CC6DF
S11312A0083734CC1008BD138BCE10091D0008304C
S11312B0C6243A35CC1D9CBD15B9CE10091D0008B5
S11312C01C0004C6083734CE10083CC6043734CC9E
S11312D01008BD138BCE10091D0004CC1DDBBD15F9
S11312E0B9CE10091D00101C0020C6103734CE10D2
S11312F0083CC6203734CC1008BD138BCE10091D12
S11313000020CC1E1ABD15B9CE10091D00201C00EA
S113131010C6203734CE10083CC6103734CC100821
S11313208D69CE10091D0010CE10261C0004CC1EA1
S113133059BD15B9CE10261D00801C0008C6803783
S113134034CE10003CC6083734CC10008D3DCE108E
S1131350261D0008CC1E98BD15B9CE10261D000808
S11313601C0080C6083734CE10003CC6803734CC0D
S113137010008D17CE10261D00801D0004CC192BE3
S1131380BD15B9308FC3001E8F35393C3CDE063C99
S1131390DE083C30ED04E60BD7096F076F06CC007E
S11313A001BD14E430EE04E6008FD6098FDD008F12
S11313B0DA01D7078FD60730EE04E70030EE0CE6EB
S11313C00030E40FE10F2767D60953D40730EE0449
S11313D0E70030EE0CE60030E50F274A30EC061A41
S11313E083000127392E18DD00270C30EC0638DF86
S11313F00838DF06383839CC1ED7BD15B920EC3093
S1131400EC061A830002270E1A83000326DDCC1E85
S1131410F0BD15B920D5CC1EF8BD15B920CDCC1F13
S11314200ABD15B920C5EC06C30002ED0620ADCCFB
S11314300001ED0620923CDE063CD707306F036FB7
S113144002CC0001BD14E4CE1000E600DA07E70088
S1131450CE1030183018E607E700E600C48027FAFB
S1131460CE1031E600C1EF2306CC000130ED02CEF0
S11314701000730007E600D407E700CE10301830E0
S113148018E607E700E600C48027FACE1031E6002C
S1131490C10F220830EC02C30002ED0230EE028CD0
S11314A0000127388F1A8300012E14DD002708302D
S11314B0EC0238DF063839CC1F1BBD15B920F030DB
S11314C0EE028C0002270D8C000326E3CC1EF0BD37
S11314D015B920DBCC1F31BD15B920D3CC1F41BDBC
S11314E015B920CBDE063C8F098CFFFF271A18CED6
S11314F0100E18EC00DD0618EC0093061A8307CFD3
S113150023F5098CFFFF26EA38DF0639CC1F51BDCD
S113151015B9CC1F87BD15B9CC07D08DC7CC1FBD5D
S1131520BD15B9CE00003CC620BD1436CC1FE7BDA6
S113153015B9CE00013CC620BD1436CC20118D79DE
S1131540CE00023CC620BD1436CC203B8D6BCE00B1
S1131550033CC620BD1436CC20658D5DCE00043C12
S1131560C640BD1436CC208F8D4FCE00053CC640FE
S1131570BD1436CC20B98D41CE00063CC640BD1406
S113158036CC20E38D33CE00073CC640BD14363044
S11315908FC300108F3539BDFFAC164F39BDFFAC7A
S11315A0810027F9164F39BDFFAC810027F9BDFF33
S11315B0B8164F3917BDFFB8398FA6002706BDFFEF
S11315C0B80820F6393617BDFFB217BDFFB532395A
S11315D036BDFFB23236BDFFB517BDFFB217BDFF32
S11315E0B532394D2A0C36862DBDFFB8324353C36C
S11315F0000118CE0000CE000A023718088F1A83A3
S1131600000026F232BDFFB5180926F83930EE0283
S11316108F1A830000270D36A600BDFFB832088359
S1131620000126F3393430E700CB9FC1192206E6C6
S113163000CBE0E700304FE60031393430E700CB2F
S1131640BFC1192206E600CB20E700304FE6003187
S1131650393CDE063CDE083CDD067F00097F0008DD
S1131660DE066D00272030ED0430EE04E6008DB573
S113167030EE04E700DE0808DF08DC06D30830EDAE
S1131680048FE60026E3DC0638DF0838DF06383945
S11316903CDE063CDE083CDD067F00097F0008DEF8
S11316A0066D00272030ED0430EE04E6008D8C300A
S11316B0EE04E700DE0808DF08DC06D30830ED049A
S11316C08FE60026E3DC0638DF0838DF06383939D0
S10416D03FD6
S11316D14465736372697074696F6E3A2054686902
S11316E1732070726F6772616D2077696C6C2074FE
S11316F1657374207468650A00706172616C6C654D
S11317016C20492F4F206665617475726573206F73
S11317116620746865203638484331312E0A000A40
S1131721005468652070726F6772616D206973205F
S113173166756C6C79206175746F6D617465642074
S1131741616E642077696C6C0A007265706F7274E3
S1131751206261636B20616E792070726F626C65C7
S11317616D7320776974682074686520492F30206F
S11317717265676973746572732E0A00496E7365C5
S113178172742074686520492F4F20546573746501
S11317917220696E746F20746865204D4355207002
S11317A16F72742077697468207468650A007369BC
S11317B16465206D61726B65642048433131206634
S11317C16163696E67207468652048433131206F15
S11317D16620746865206576616C756174696F6EE5
S11317E120626F6172642E0A0021212121212121AD
S11317F1212121215645525920494D504F525441DE
S11318014E54205245414420544845205354415498
S1131811454D454E542042454C4F5721212121210C
S113182121212121212121212121210A0A004D41A6
S11318314B45205355524520594F5520444F204E76
S11318414F54204841564520414E59204F54484554
S11318515220434F4D504F4E454E54530A00434F6F
S11318614E4E454354454420544F2054484520503E
S11318714152414C4C454C20492F4F2050494E5325
S1131881204F4620544845204556414C5541544922
S11318914F4E20424F4152440A0A00212121212165
S11318A12121212121215645525920494D504F5280
S11318B154414E54205245414420544845205354E8
S11318C14154454D454E542041424F5645204147D0
S11318D141494E212121212121212121210A005780
S11318E168656E2074686520746573746572206917
S11318F1732070726F7065726C7920696E73657292
S11319017465642C2063686F6F7365206F6E652046
S11319116F662074686520666F6C6C6F77696E679B
S1131921206F7074696F6E733A000A0A004F707405
S1131931696F6E730A002D2D2D2D2D2D2D2D2D0A40
S11319410020413A2041444320546573740A002025
S1131951503A20506172616C6C656C20492F4F20A4
S1131961546573740A0020453A20546573742062E7
S11319716F74682041444320616E64205061726138
S11319816C6C656C20492F4F0A0020513A20517527
S113199169740A0050726F6772616D206973206EF9
S11319A16F77207465726D696E6174696E672E2E2E
S11319B12E2E2E2E2E2E2E2E2E2E2E2E2E2E2E2E42
S11319C12E2E2E0A004E6F772074657374696E672C
S11319D1207374616E6461726420696E70757473CE
S11319E120616E64206F7574707574732C20706C33
S11319F16561736520776169742E2E2E2E2E0A007F
S1131A012D2D2D2D2D2D2D2D2D2D2D2D2D2D2D2D01
S1131A112D2D2D2D2D2D2D2D2D2D2D2D2D2D2D2DF1
S1131A212D2D2D2D2D2D2D2D2D2D2D2D2D2D2D2DE1
S1131A312D2D2D2D2D2D0A0A0054657374696E67A1
S1131A413A20504134202D3E20504130202E2E2E5C
S1131A512E2E2E2E2E2E2E2E2E2E2E2E2E2E2E2EA1
S1131A612E2E2E2E2E2E2E2E2E2E2E2E2E2E2E2E91
S1131A712E2E2E2E2E2E2E0054657374696E673A07
S1131A8120504134202D3E20504131202E2E2E2E27
S1131A912E2E2E2E2E2E2E2E2E2E2E2E2E2E2E2E61
S1131AA12E2E2E2E2E2E2E2E2E2E2E2E2E2E2E2E51
S1131AB12E2E2E2E2E2E0054657374696E673A20D5
S1131AC1504134202D3E20504132202E2E2E2E2ED8
S1131AD12E2E2E2E2E2E2E2E2E2E2E2E2E2E2E2E21
S1131AE12E2E2E2E2E2E2E2E2E2E2E2E2E2E2E2E11
S1131AF12E2E2E2E2E0054657374696E673A205073
S1131B014135202D3E20504530202E2E2E2E2E2EB6
S1131B112E2E2E2E2E2E2E2E2E2E2E2E2E2E2E2EE0
S1131B212E2E2E2E2E2E2E2E2E2E2E2E2E2E2E2ED0
S1131B312E2E2E2E0054657374696E673A2050411F
S1131B4135202D3E20504531202E2E2E2E2E2E2E88
S1131B512E2E2E2E2E2E2E2E2E2E2E2E2E2E2E2EA0
S1131B612E2E2E2E2E2E2E2E2E2E2E2E2E2E2E2E90
S1131B712E2E2E0054657374696E673A20504135D8
S1131B81202D3E20504532202E2E2E2E2E2E2E2E4E
S1131B912E2E2E2E2E2E2E2E2E2E2E2E2E2E2E2E60
S1131BA12E2E2E2E2E2E2E2E2E2E2E2E2E2E2E2E50
S1131BB12E2E0054657374696E673A2050413520A6
S1131BC12D3E20504533202E2E2E2E2E2E2E2E2EFF
S1131BD12E2E2E2E2E2E2E2E2E2E2E2E2E2E2E2E20
S1131BE12E2E2E2E2E2E2E2E2E2E2E2E2E2E2E2E10
S1131BF12E0054657374696E673A20504136202D66
S1131C013E20504534202E2E2E2E2E2E2E2E2E2EBC
S1131C112E2E2E2E2E2E2E2E2E2E2E2E2E2E2E2EDF
S1131C212E2E2E2E2E2E2E2E2E2E2E2E2E2E2E2ECF
S1131C310054657374696E673A20504136202D3E15
S1131C4120504535202E2E2E2E2E2E2E2E2E2E2E8B
S1131C512E2E2E2E2E2E2E2E2E2E2E2E2E2E2E2E9F
S1131C612E2E2E2E2E2E2E2E2E2E2E2E2E2E2E00BD
S1131C7154657374696E673A20504136202D3E20B5
S1131C81504536202E2E2E2E2E2E2E2E2E2E2E2E3C
S1131C912E2E2E2E2E2E2E2E2E2E2E2E2E2E2E2E5F
S1131CA12E2E2E2E2E2E2E2E2E2E2E2E2E2E005457
S1131CB1657374696E673A20504136202D3E205079
S1131CC14537202E2E2E2E2E2E2E2E2E2E2E2E2E1D
S1131CD12E2E2E2E2E2E2E2E2E2E2E2E2E2E2E2E1F
S1131CE12E2E2E2E2E2E2E2E2E2E2E2E2E004E6FDC
S1131CF1772074657374696E6720746865206269FE
S1131D012D646972656374696F6E616C2070696EAC
S1131D11732C20706C6561736520776169742E2E54
S1131D212E2E2E0A002D2D2D2D2D2D2D2D2D2D2D2B
S1131D312D2D2D2D2D2D2D2D2D2D2D2D2D2D2D2DCE
S1131D412D2D2D2D2D2D2D2D2D2D2D2D2D2D2D2DBE
S1131D512D2D2D2D2D2D2D2D2D0A0A005465737435
S1131D61696E673A20504433202D3E20504432207E
S1131D712E2E2E2E2E2E2E2E2E2E2E2E2E2E2E2E7E
S1131D812E2E2E2E2E2E2E2E2E2E2E2E2E2E2E2E6E
S1131D912E2E2E2E2E2E2E2E2E2E00546573746969
S1131DA16E673A20504432202D3E20504433202E79
S1131DB12E2E2E2E2E2E2E2E2E2E2E2E2E2E2E2E3E
S1131DC12E2E2E2E2E2E2E2E2E2E2E2E2E2E2E2E2E
S1131DD12E2E2E2E2E2E2E2E2E0054657374696EE9
S1131DE1673A20504435202D3E20504434202E2E75
S1131DF12E2E2E2E2E2E2E2E2E2E2E2E2E2E2E2EFE
S1131E012E2E2E2E2E2E2E2E2E2E2E2E2E2E2E2EED
S1131E112E2E2E2E2E2E2E2E0054657374696E676F
S1131E213A20504434202D3E20504435202E2E2E6D
S1131E312E2E2E2E2E2E2E2E2E2E2E2E2E2E2E2EBD
S1131E412E2E2E2E2E2E2E2E2E2E2E2E2E2E2E2EAD
S1131E512E2E2E2E2E2E2E0054657374696E673A23
S1131E6120504133202D3E20504137202E2E2E2E3E
S1131E712E2E2E2E2E2E2E2E2E2E2E2E2E2E2E2E7D
S1131E812E2E2E2E2E2E2E2E2E2E2E2E2E2E2E2E6D
S1131E912E2E2E2E2E2E0054657374696E673A20F1
S1131EA1504137202D3E20504133202E2E2E2E2EF0
S1131EB12E2E2E2E2E2E2E2E2E2E2E2E2E2E2E2E3D
S1131EC12E2E2E2E2E2E2E2E2E2E2E2E2E2E2E2E2D
S1131ED12E2E2E2E2E00486967682026206C6F77DF
S1131EE1207465737473206661696C65640A0050BB
S1131EF161737365640A0048696768207465737463
S1131F01206661696C65640A004C6F77207465739F
S1131F1174206661696C65640A0035562026203098
S1131F2156207465737473206661696C65640A0074
S1131F3135562074657374206661696C65640A00A2
S1131F4130562074657374206661696C65640A0097
S1131F514E6F772074657374696E672074686520A9
S1131F61412F4420636F6E766572746572207069C7
S1131F716E732C20706C6561736520776169742EB2
S1131F812E2E2E2E0A002D2D2D2D2D2D2D2D2D2DC8
S1131F912D2D2D2D2D2D2D2D2D2D2D2D2D2D2D2D6C
S1131FA12D2D2D2D2D2D2D2D2D2D2D2D2D2D2D2D5C
S1131FB12D2D2D2D2D2D2D2D2D0A0A0054657374D3
S1131FC1696E673A20504135202D3E20504530201E
S1131FD12E2E2E2E2E2E2E2E2E2E2E2E2E2E2E2E1C
S1131FE12E2E2E2E2E0054657374696E673A20507E
S1131FF14135202D3E20504531202E2E2E2E2E2EC1
S11320012E2E2E2E2E2E2E2E2E2E2E2E2E2E2E0019
S113201154657374696E673A20504135202D3E2012
S1132021504532202E2E2E2E2E2E2E2E2E2E2E2E9C
S11320312E2E2E2E2E2E2E2E2E0054657374696E86
S1132041673A20504135202D3E20504533202E2E15
S11320512E2E2E2E2E2E2E2E2E2E2E2E2E2E2E2E9B
S11320612E2E2E0054657374696E673A20504136E2
S1132071202D3E20504534202E2E2E2E2E2E2E2E57
S11320812E2E2E2E2E2E2E2E2E2E2E2E2E0054653C
S11320917374696E673A20504136202D3E205045B5
S11320A135202E2E2E2E2E2E2E2E2E2E2E2E2E2E52
S11320B12E2E2E2E2E2E2E0054657374696E673AC1
S11320C120504136202D3E20504536202E2E2E2ED6
S11320D12E2E2E2E2E2E2E2E2E2E2E2E2E2E2E2E1B
S11320E12E0054657374696E673A20504136202D71
S11320F13E20504537202E2E2E2E2E2E2E2E2E2EC5
S10F21012E2E2E2E2E2E2E2E2E2E2E00D4
S104210D00CD
S9031040AC
